:020000040000FA
:100000000313831200308B0000308500003086001F
:1000100007309F008316C530810010308500F03016
:10002000860083120030A800A90085150511A801DB
:10003000A901A601A701B601B701B801AA30A00025
:10004000A61113221322132233300222333002224C
:10005000323002222C300222063002220C300222E0
:100060000130022202300222132213220130EE223A
:10007000A20006148511061E3F280130A206861E26
:100080004328A2142211061F47282215A210861FFA
:100090004B282211A21085150610DA22A218722808
:1000A00022197A2801224C3003224F300322433098
:1000B0000322203003225330032250300322203009
:1000C0000322443003222030032231300322323015
:1000D00003223330032234300322203003224630FF
:1000E00003228C280122543003224F300322473050
:1000F0000322592801224C3003224F3003224B3077
:1001000003222030032246300322533003222030C2
:100110000322523003226328DE201021292153219B
:10012000A321FB219E20C9209E20C920C920AF0DFC
:10013000AF1E8C28AF0103102F148C283E08AA0094
:100140000830A4000510AA0DD820031C0514CF20E8
:100150000514D820A40BA2280510D820A71E05142A
:10016000CF200514D8200510D820271F0514CF2034
:100170000514D8202108AA000830A4000510AA0DF3
:10018000D820031C0514CF200514D820A40BBE28AA
:1001900008002630A3002921A30BCB280800053036
:1001A000A3000000000000002921A30BD4280800B0
:1001B0000430A3000000A30BDA280800C622221C8A
:1001C000FF2122180122303003222808303E03226A
:1001D0002908303E032220300322250803223D084F
:1001E0000322203003223C302718023E0322203015
:1001F00003222030A7180A3E0322203027190A3E86
:1002000003222030A7190A3E03222030271A0A3E73
:100210000322203003222030A71A0A3E03220800BE
:100220008511AB010430AC0086010314860D031068
:10023000061A2629AB0A861A2629AB0A061B262986
:10024000AB0A861B2629AB0AAC0B1629851586013D
:1002500008003810B81085150608C039B600031913
:10026000B814370203193814C03036020319B81411
:10027000B81C432938184C29381DAE0A3819AE036A
:100280003608B700080038113708B606B61B38150F
:100290000000000000000800000000000000000056
:1002A0000000000008002B1A9F292B08083EEE22B0
:1002B000AB000A302B0203187129261908002618F2
:1002C00069292614A6142B08A8007030A9003A2228
:1002D0000800A618080026102B08A90026151C22C5
:1002E0000800A619A029A6150B302B02031D7C2996
:1002F000AE010130A706A0290A302B02031D832975
:100300002030A706A0290C302B02031D8A290230B9
:10031000A706A0290D302B02031D91290430A70642
:10032000A0290E302B02031D98290830A706A0290A
:100330000F302B02031DA0291030A706A029A611FB
:10034000A61026110800A61DAC290B302B02031D98
:10035000AC29C030A1000800B00103102F1CB42943
:10036000271CB4291030B000AF1CBA292030A718C0
:100370006030B0002F1DC029303027197030B00018
:10038000AF1DC6294030A7198030B0002F1ECC29E0
:100390005030271A9030B000C0302E020318AE0142
:1003A0001C302E02031CD6291C30AE0003112E0374
:1003B000031DDD290430AE00E129FD302E070319AD
:1003C000AE012E08B9003918EC29B90CB913A71AD7
:1003D0002717A71E2713F229B90CB913A71A271339
:1003E000A71E27173908B00703308A0030080023FA
:1003F0008A01A1000800051E08002921FB29C03040
:10040000022A80308511B4001430B300B30B062AE1
:100410000C220C2285150800B40E34080F39860012
:100420000515051108000A30B5008B010B1D162AB1
:100430000B11B50B162A0800BF012808B1000310E4
:10044000310DB10EB10C31072907A000AD003230DB
:100450002D02031C2F2A0230BF003230AD020310E0
:10046000AD0DAD0DB1221F302E02031C0800AE01F0
:10047000A7010800BF012008AD0032302D02031C87
:10048000452A0230BF003230AD020310AD0DAD0D74
:10049000A522080083168514831208008510831690
:1004A0008510831208000614080006100800532265
:1004B00000000000000000005522000000000000C5
:1004C0000000080055224A2253224E2255220000E5
:1004D000000000000000080055224E2253224A224C
:1004E0005522000000000000000008004A225722A8
:1004F00008004E2257220800BB000830BA00031043
:10050000BB0D0318872A4E2257224A22892A4A22E3
:100510005722BA0B7F2A762208000830BA004A22F6
:10052000532200000000000000000000851C9A2AF1
:1005300003149B2A0310BC0D55220000000000008C
:100540000000BA0B902A3C0808006222A0303F0746
:100550007C222D087C222E087C2227087C226C22FB
:1005600008006222A0303F077C222D087C226222F4
:10057000A1303F077C228D22AE0079228D22A70078
:1005800079228D22BE0076226C22080003112E08EB
:10059000031DFD3EB200B1010A303202031CD32A12
:1005A000B200B10ACC2A3108303EA5003208303EF4
:1005B000BD000800220883169A0001309B008B13AF
:1005C0001C129C111C1555309D00AA309D009C14D6
:1005D0001C119C18E92A83128B17080083169B00B4
:0805E0001C141A088312080024
:100600008207113491343134B13419349934393486
:10061000B934123492343234B2341A349A343A340B
:10062000BA344534C5346534E5344D34CD346D3495
:10063000ED344634C6346634E6344E34CE346E344B
:10064000EE345034D0347034E4345834D834783400
:10065000F8345234D2347234F2345A34DA347A34CC
:10066000FA34043484342434A4344C348C342C349C
:10067000AC34063486342634A6340E348E342E340C
:10068000AE34143494343434B4341C349C346C3468
:10069000BC34163496343634B6341E349E343E346C
:1006A000BE345434D4347434F4345C34DC347C34A8
:1006B000EC345634D6347634F6345E34DE347E345C
:1006C000FE345134D1347134F1345934D93479345D
:1006D000F9345334D3347334B3345B34DB347B3484
:1006E000FB34053485342534A5340D348D342D3454
:1006F000AD34073487342734A7341B348F342F3478
:10070000AF34153495343534B5341D349D343D340F
:10071000BD34173497343734B7341F349F343B34E7
:10072000BF345534D5347534F5345D34DD347D341F
:10073000FD345734D7347734F7345F34DF347F34C3
:02074000BB34C8
:02400E00383F39
:1042000000000000000000000000000000000000AE
:104210000100020003000F000400050006000E006C
:104220000700080009000D000A0000000B000C0048
:10423000000000000000000000000000000000007E
:10424000000000000000000000000000000000006E
:10425000000000000000000000000000000000005E
:10426000000000000000000000000000000000004E
:10427000000000000000000000000000000000003E
:00000001FF
